:020000040000FA
:100000002E288207003400340034003400341B34BE
:1000100077344034003435346734E03400346A34A3
:10002000CF34C03400349A341D3420340034D534F5
:100030009F34803401341334B234203401344034DA
:100040006F34403401347B34CA3490340134AB34DF
:100050003F3400340134C934C33480348B01073059
:100060009F00C22383168113FF308500860183120F
:10007000AD01AE01AF01B001B101E622E622CA2016
:10008000EA20D201051A4728521422225210831660
:100090009B01AA231A088312BB008316AA231A08FD
:1000A0008312BC008316AA231A088312BD0083168C
:1000B000AA231A088312BE008316AA231A088312E1
:1000C000A0008316AA231A088312A1008316AA236C
:1000D0001A088312A2008316AA231A088312A30007
:1000E00000232E23AF22E6220508CB0003304B0568
:1000F000CA00CC01D001A5214B1A8028A0207B2862
:10010000B501B401B301D2198A28521A8F280130DF
:10011000B2009528E830B2000330B30095280F30C4
:10012000B4004230B3004030B200CC18992892217C
:100130009B2855216D2100232E23AF22E6227B2808
:10014000CC18AC280430D002D7305007031CAA28A2
:100150002830D000B820B3280430D007D73050075B
:100160000318D001B82000232E23AF22E622080076
:1001700050080120A300D00A50080120A200D00A94
:1001800050080120A100D00A50080120A00003302F
:10019000D0020800B923033086000616B9230612E0
:1001A000033086000616BC230612033086000616AE
:1001B000BC230612023086000616BF230612283022
:1001C0007B2308307B2301307B2306307B230C30DC
:1001D0007B23080080307B2350307F2349307F23EE
:1001E00043307F2345307F234C307F2367307F238C
:1001F00065307F236E307F238830C3007B23373008
:100200007F232E307F2332307F232D307F233630E3
:100210007F2330307F2320307F2320307F23C03066
:100220007B2350307F2349307F2343307F23473067
:100230007F2345307F234E307F2320307F2337308C
:100240007F232E307F2332307F2320307F232030C6
:100250007F2320307F2320307F2320307F232030D6
:100260007F23AE23C0307B2353307F2354307F2342
:1002700045307F2350307F233A307F2331307F2336
:1002800048307F237A307F2320307F2320307F2324
:1002900020307F2320307F2320307F2320307F2396
:1002A00020307F2320307F2308003208A007031C62
:1002B0005E29A10F5E29A20F5E29A30A3308A107B8
:1002C000031C6529A20F6529A30A3408A207031C91
:1002D0006A29A30A3508A3070800FC30230703187E
:1002E000892903302302031C91296C30220703184B
:1002F000892993302202031C9129783021070318A1
:10030000892987302102031C912900302002031C17
:1003100091290030A0008730A1009330A200033063
:10032000A3000800B209B309B409B509B20F9D29A9
:10033000B30F9D29B40F9D29B50A5521A31FA429E8
:10034000A001A101A201A3010800521CD3210508AC
:10035000CB00C42305084B06031DA52903304B051C
:10036000C9004A060319A5290310CA0D4908CA067F
:100370004A080239CD004C06CC01CA18C7294908E1
:10038000CA00CF034F18A529CF18A529D0290230BC
:10039000CC004908CA00CF0A4F18A529CF18A529B3
:1003A0004908CA0008008519FC29C2238519FC29BF
:1003B000D21DE629D21100005216C6307B234D30E3
:1003C0007F2348307F237A307F231F2A521AF22955
:1003D000D215C6307B236B307F2348307F237A30A1
:1003E0007F231F2A5212C6307B2348307F237A3066
:1003F0007F2320307F231F2A05191F2A1030D300A6
:1004000005191F2AB623D30B002A9622CB307B2353
:1004100053307F2341307F2356307F2345307F2365
:1004200044307F23AE23CB307B2320307F2320300A
:100430007F2320307F2320307F2320307F23851DA2
:100440001F2A08008030A0009630A1009830A2003A
:100450000030A30083169B01AA231A088312BB0055
:100460008316AA231A088312BC008316AA231A082B
:100470008312BD008316AA231A088312BE0000232C
:100480002E23C430C3007B234330C3007F2341307D
:10049000C3007F234C30C3007F23AF22E622A52177
:1004A000B501B401B3011030B2004B19592A8030A4
:1004B000B2000000CC18672AB209B309B409B50923
:1004C000B20F672AB30F672AB40F672AB50A32083A
:1004D000BB07031C702ABC0F702ABD0F702ABE0A0E
:1004E0003308BC07031C772ABD0F772ABE0A3408DD
:1004F000BD07031C7C2ABE0A3508BE07051E4D2A0F
:100500003B0883169B019A009D2383123C088316A7
:100510009A009D2383123D0883169A009D2383121F
:100520003E0883169A009D23831208008316043028
:100530009B008312200883169A009D2383122108B2
:1005400083169A009D238312220883169A009D2306
:100550008312230883169A009D2383120800AD019D
:10056000AE01AF01B001B1012030B8003B08BF00BF
:100570003C08C0003D08C1003E08C20003103F1CFB
:10058000D82A2008AE07031CCA2AAF0FCA2AB00F08
:10059000CA2AB10A2108AF07031CD12AB00FD12AF9
:1005A000B10A2208B007031CD62AB10A2308B107F2
:1005B000B10CB00CAF0CAE0CAD0CC20CC10CC00C2D
:1005C000BF0CB80BBE2A0130B10008002D308400EA
:1005D0000008BA000830B900BA0C031CF32A8615CB
:1005E00006150611F62A861106150611B90BEC2A16
:1005F000840A32300402031CE82A86178613080096
:100600002030B600A801A901AA01AB01AC0103107A
:10061000A00DA10DA20DA30D03182014A80DA90D66
:10062000AA0DAB0DAC0DB603031D172B0800283027
:1006300084002323840A2323840A2323840A232374
:10064000840A2323072B03300007B700B719800063
:1006500030300007B700B71B8000080080307B23D4
:1006600020307F232B0E0F39303E7F232B080F398C
:10067000303E7F232C307F232A0E0F39303E7F23DC
:100680002A080F39303E7F23290E0F39303E7F2351
:100690002E307F2388307B2329080F39303E7F237B
:1006A000280E0F39303E7F2328080F39303E7F2334
:1006B00020307F236B307F2348307F237A307F23A5
:1006C00020307F23080086018316083086008312BD
:1006D00006138616FF30C50006160608C40006126B
:1006E00000000000061600000612C50303197A2B4D
:1006F000C4196C2B0800C300D1010613822BC30060
:100700005114061763238601831600308600831276
:100710008612061351180617F0308605430E0F395E
:100720008604061600000612F030860543080F39CD
:10073000860406160000061208001C158B1355309F
:100740009D00AA309D009C149C18A42B9C171C1182
:100750009B0A08001C141A089B0A0800B323B32341
:10076000B323B3230800B623B6230800FF30C50027
:10077000C62B8030C500C62B4030C500C62B2030AC
:10078000C500C62B1030C5000230C500FF30C600C2
:0A079000C60BC82BC50BC62B0800D2
:02400E00303F41
:10420000DE006500DC00170028000100D600000079
:10421000000000000000000000000000000000009E
:10422000000000000000000000000000000000008E
:10423000000000000000000000000000000000007E
:10424000000000000000000000000000000000006E
:10425000000000000000000000000000000000005E
:10426000000000000000000000000000000000004E
:10427000000000000000000000000000000000003E
:10428000000000000000000000000000000000002E
:10429000000000000000000000000000000000001E
:1042A000000000000000000000000000000000000E
:1042B00000000000000000000000000000000000FE
:1042C00000000000000000000000000000000000EE
:1042D00000000000000000000000000000000000DE
:1042E00000000000000000000000000000000000CE
:00000001FF
